:100000000C9446000C9463000C9463000C94630001
:100010000C9463000C9463000C9463000C946300D4
:100020000C9463000C9463000C9463000C946300C4
:100030000C9463000C9463000C9463000C946300B4
:100040000C9463000C9463000C9463000C946300A4
:100050000C9463000C9463000C9463000C94630094
:100060000C9463000C9463000C9463000C94630084
:100070000C9463000C9463000C9463000C94630074
:100080000C9463000C9463000C94630011241FBE55
:10009000CFEFD0E1DEBFCDBF11E0A0E0B1E0E8E1FD
:1000A000F3E000E00BBF02C007900D92A030B10753
:1000B000D9F711E0A0E0B1E001C01D92A030B10776
:1000C000E1F70C9465000C940000CDEFD0E1DEBFA9
:1000D000CDBF89ED8093370084E68093530083E69B
:1000E000809345001A8219820E9476010E94820143
:1000F0000E941D010E9482010E9476010E948201DD
:100100000E943C010E9482010E9476010E948201AD
:100110000E941D010E9482010E9476010E948201BC
:100120000E941D010E9482010E9476010E948201AC
:100130000E943C010E94820180E090E00C948B01BF
:10014000CF93DF93CDB7DEB724970FB6F894DEBF19
:100150000FBECDBF19821A821B821C8289819A81AF
:10016000AB81BC81803523EC920720E0A20720E020
:10017000B20764F489819A81AB81BC810196A11D8B
:10018000B11D89839A83AB83BC83E8CF24960FB6D5
:10019000F894DEBF0FBECDBFDF91CF910895CF930E
:1001A000DF93CDB7DEB722970FB6F894DEBF0FBE50
:1001B000CDBF10925100109243001A82198289819A
:1001C0009A818431910594F480915100865F8093E7
:1001D000510080914300865F809343000E94A000FD
:1001E00089819A8101969A838983E9CF22960FB6F5
:1001F000F894DEBF0FBECDBFDF91CF910895CF93AE
:10020000DF93CDB7DEB780915100809151008531E9
:1002100068F0809151008A50809351008091430092
:100220008A50809343000E94A000EFCF10925100AB
:1002300010924300DF91CF910895CF93DF93CDB714
:10024000DEB781E4809338008091510080915100A5
:100250008C3868F480915100865F809351008091C2
:100260004300865F809343000E94A000EFCF0E946E
:10027000A000DF91CF910895CF93DF93CDB7DEB784
:1002800089E08093380080915100809151008E3632
:1002900068F480915100865F809351008091430003
:1002A000865F809343000E94A000EFCFDF91CF9143
:1002B0000895CF93DF93CDB7DEB781E48093380004
:1002C00080915100809151008E3668F480915100E8
:1002D000865F8093510080914300865F8093430046
:1002E0000E94A000EFCFDF91CF910895CF93DF93CD
:1002F000CDB7DEB781E0809338000E94CF00DF9158
:10030000CF910895CF93DF93CDB7DEB70E94FF0062
:08031000DF91CF910895FFCFAA
:00000001FF
